:020000021000EC
:04E800000C9400F87C
:10E8100084B7877F84BF88E10FB6F8948093600047
:10E82000109260000FBE90E080E80FB6F8948093DD
:10E830006100909361000FBEC1E0C5BF82E085BF5B
:10E84000C3D6C0936F0083E0809381007894809159
:10E850000001882339F081E091E00E9476FD0E945A
:10E86000FFFCF5CF8091800291E0980F9093800299
:10E870008F3F89F78091E00081608093E00082E41F
:10E880009CED90938C0280938B022CE088E190E0C9
:10E890000FB6F894A895809360000FBE2093600097
:10E8A000FFCF0895089581E091E00C9459FD81E037
:10E8B00091E00C941AFD70D010928002089591306E
:10E8C00039F0923051F080E090E020E030E009C073
:10E8D00082E190E02CE032E004C080E290E02CEE97
:10E8E00031E0FA013183208308959F92AF92BF9265
:10E8F000CF92DF92EF92FF920F931F93CF93DF930C
:10E90000EC01962EC8A0DF8CABA0BAA08CE1C81693
:10E9100081E0D80618F400E010E015C080913C01B9
:10E92000807F856080933C0181E280934601109254
:10E93000470180E025C0C8018C0D9D1D992039F04C
:10E9400003D20F5F1F4F0A151B05A9F702C032D172
:10E95000F8CF6801E12CF12C89E0CC0CDD1CEE1C19
:10E96000FF1C8A95D1F74C895D896E897F894C1986
:10E970005D096E097F094C8B5D8B6E8B7F8B81E00F
:10E98000DF91CF911F910F91FF90EF90DF90CF908B
:10E99000BF90AF909F900895EF92FF920F931F93B7
:10E9A000CF93DF93EC018B8D8F31A0F48D3108F084
:10E9B000C0C08231F1F138F4882309F4BAC0833041
:10E9C00009F468C0BBC08A3109F491C08B3109F4E5
:10E9D000A8C0B4C0883209F483C020F5853209F09C
:10E9E000ADC01092F1001092F10081E08093F1002F
:10E9F0008BE18093F1001092F1001092F10082E01F
:10EA00008093F1001092F1008091E8008E7780935E
:10EA1000E8004C895D896E897F89485051096109F8
:10EA200071097AC08A3209F459C08F3209F481C061
:10EA300085C00F8D1E8D8C8D837019F48D8D88236C
:10EA400041F080913C01807F856080933C0184E2AD
:10EA50007CC078010532110518F024E2E22EF12C79
:10EA600040E050E0B7018EE192E0E6D360E070E074
:10EA7000C8018E199F09A3D38091E8008E778093F7
:10EA8000E8004C895D896E897F894E195F096109AB
:10EA9000710942C0EF8CFE2C82E18E1510F492E1D8
:10EAA000F92E0F2D10E040E050E0B8018AE391E02C
:10EAB000C3D38E2D90E060E070E0801B910B7FD37C
:10EAC0008091E8008E778093E8004C895D896E899B
:10EAD0007F894F195109610971091EC060E001C0A9
:10EAE00061E0CE0102DF882309F43FC033C01092F9
:10EAF000F1001092F1001092F1001092F10080915B
:10EB0000E8008E778093E8004C895D896E897F8963
:10EB100044505109610971094C8B5D8B6E8B7F8B61
:10EB200019C08F8D837091E0823009F490E090934A
:10EB300000011C8A1D8A1E8A1F8A0CC080913C011C
:10EB4000807F856080933C0180E280934601109233
:10EB500047010BC080913C01807F80933C01109263
:10EB600046011092470181E001C080E0DF91CF9122
:10EB70001F910F91FF90EF900895FB01F695E79597
:10EB8000E60FF0E0E80FF91F60FF0EC080818F7084
:10EB9000942F9295907F892B808384E0569547959A
:10EBA0008A95E1F7418308954083842F807F852BE8
:10EBB000818308954F925F926F927F928F929F927E
:10EBC000AF92BF92CF92DF92EF92FF920F931F937B
:10EBD000CF93DF93CDB7DEB7D2500FB6F894DEBF38
:10EBE0000FBECDBF8C0140E050E060E072E0CE018E
:10EBF000019669D38091E8008B778093E800033019
:10EC0000110508F48AC00330110551F480EAFE01B1
:10EC10003196ACE4B1E001900D928A95E1F77DC0A8
:10EC20008091A6019091A7018150904C880F991F67
:10EC3000880F991F0817190778F48091E6019091C1
:10EC4000E7018150904C880F991F880F991F081772
:10EC5000190708F044C061C09C012D503F4F201798
:10EC6000310758F36801C81AD90AE12CF12C79E070
:10EC7000CC0CDD1CEE1CFF1C7A95D1F7CE01019661
:10EC80005C014E019FEF891A9DEF990AC11003C0E4
:10EC9000C701B6013AD2F501418150E0542F442713
:10ECA0008081482BC701B60158D226013701F2E016
:10ECB0004F0E511C611C711C411007C0C701B601E9
:10ECC0006E5F71098109910934D282E0A80EB11CEE
:10ECD000A814B90409F4B1CF73016201D7CF9C0124
:10ECE000295F3F4F20173107C0F0081B190B102F69
:10ECF0000027110FFE0131966F01E12CF12CF60176
:10ED000061916F01C701800F911F58D2FFEFEF1A79
:10ED1000FF0AE11482E0F80691F7DE5F0FB6F8947F
:10ED2000DEBF0FBECDBFDF91CF911F910F91FF903E
:10ED3000EF90DF90CF90BF90AF909F908F907F909B
:10ED40006F905F904F900895AF92BF92CF92DF92F5
:10ED5000EF92FF920F931F93CF93DF93CDB7DEB760
:10ED6000C150D2400FB6F894DEBF0FBECDBF8E01AA
:10ED70000F5F1F4F20E032E0F801A90111924150CE
:10ED80005040E1F783309105B8F4019710F58EE318
:10ED9000E2E4F2E0D80101900D928A95E1F785E571
:10EDA000C150DE4F8883CF5FD1408AEAC050DE4F2A
:10EDB0008883C050D240A8C08330910509F044C078
:10EDC00080EAECE4F1E0D80101900D928A95E1F738
:10EDD0009BC048EF5FE060E070E0C801CEDE4FEF1F
:10EDE0005FE061E070E0C801C8DE6091A60170914B
:10EDF000A70120E0CB0101967C012C3311F0AC017E
:10EE000002C04FEF5FE0C801CF5FDD4F2883C150E4
:10EE1000D240B3DECF5FDD4F2881C150D2402F5F9B
:10EE2000B7012D3339F76091E6017091E7017B015D
:10EE30009FEFE91AF90AA701C8019FDE4FEF5FE0D3
:10EE4000B701C8019ADE60C02091A6013091A701E8
:10EE50002150304C220F331F220F331F821793078C
:10EE600070F42091E6013091E7012150304C220FDF
:10EE7000331F220F331F8217930740F545C0A901A6
:10EE80004D505F4F4817590760F3AC01421B530BBD
:10EE900060E070E0B9E0440F551F661F771FBA9518
:10EEA000D1F7D8019E012F5F3D4F6A017B01EFEF43
:10EEB000CE1ADE0AEE0AFE0A6BBFFA0147914D93A5
:10EEC000A217B30771F2B701A601EFCFA901495FFD
:10EED0005F4F48175907C0F07C01E21AF30AFE2C75
:10EEE000EE24FF0C5E01FFEFAF1AFDEFBF0A6801D1
:10EEF000E01AF10AC7018C0D9D1D5FD1F6018193C7
:10EF00006F01EA15FB05B1F740E050E060E072E008
:10EF1000C80192D18091E8008E778093E800CF5F9E
:10EF2000DD4F0FB6F894DEBF0FBECDBFDF91CF919E
:10EF30001F910F91FF90EF90DF90CF90BF90AF9017
:02EF4000089532
:10F000004BC0000077C0000075C0000073C0000056
:10F0100071C000006FC000006DC000006BC0000038
:10F0200069C0000067C00000EAC20000A4C300007D
:10F0300061C000005FC000005DC000005BC0000058
:10F0400059C0000057C0000055C0000053C0000068
:10F0500052C000004FC000004DC000004BC0000077
:10F0600049C0000047C0000045C0000043C0000088
:10F0700041C000003FC000003DC000003BC0000098
:10F0800039C0000037C0000035C0000033C00000A8
:10F0900031C000002FC0000011241FBECFEFD0E20E
:10F0A000DEBFCDBF04B603FE0EC080918B029091EF
:10F0B0008C0282349C4D39F410928C0210928B0297
:10F0C000E0E0F0E0099512E0A0E0B1E0E2E5FDEF5C
:10F0D00001E00BBF02C007900D92A038B107D9F72D
:10F0E00022E0A0E8B2E001C01D92AB38B207E1F720
:10F0F0008FDB2DC685CF1F920F920FB60F92112472
:10F100000F900FBE0F901F90189507B600FCFDCF13
:10F11000F999FECF23E0FB0180935B002093570019
:10F12000E89507B600FCFDCF81E180935700E89594
:10F13000089507B600FCFDCFF999FECF25E0FB014D
:10F1400080935B0020935700E89507B600FCFDCF45
:10F1500081E180935700E895089507B600FCFDCF44
:10F16000F999FECF21E00A01FB0180935B00209317
:10F170005700E8951124089521E2FC0120935700DF
:10F180008491089529E0FC0120935700849108950B
:10F19000E1E0F0E089E0809357008491089507B69C
:10F1A00000FCFDCFF999FECF809599E0E1E0F0E019
:10F1B000082E90935700E8950895AFC5B6C5EF9215
:10F1C000FF920F931F93CF93DF938C01EB018DD1AF
:10F1D00081112BC0209721F088819981081B190B80
:10F1E000E12CF12C01151105F9F08091E80085FD65
:10F1F00013C08091E8008E778093E800209741F05B
:10F20000888199818E0D9F1D9983888385E00DC02B
:10F210006CD1882339F309C01092F1000150110913
:10F220008FEFE81AF80ADECF80E0DF91CF911F91CF
:10F230000F91FF90EF900895CF92DF92EF92FF929F
:10F240000F931F93CF93DF937C018B01EA014DD184
:10F25000811130C0209731F088819981081B190BEA
:10F26000E80EF91EC12CD12C0115110511F1809168
:10F27000E80085FD13C08091E8008E778093E80058
:10F28000209741F0888199818C0D9D1D99838883F9
:10F2900085E010C02AD1882339F30CC0F701819191
:10F2A0007F018093F10001501109FFEFCF1ADF0AAF
:10F2B000DBCF80E0DF91CF911F910F91FF90EF9016
:10F2C000DF90CF900895CF92DF92EF92FF920F934D
:10F2D0001F93CF93DF937C018B01EA0106D181114B
:10F2E00030C0209731F088819981081B190BE80EF6
:10F2F000F91EC12CD12C0115110511F18091E800E6
:10F3000085FD13C08091E8008B778093E8002097FB
:10F3100041F0888199818C0D9D1D9983888385E0BA
:10F3200010C0E3D0882339F30CC08091F100F701BD
:10F3300081937F0101501109FFEFCF1ADF0ADBCF64
:10F3400080E0DF91CF911F910F91FF90EF90DF90C0
:10F35000CF9008952091890230918A0226173707AD
:10F3600048F06115710539F42091E8002E7720935B
:10F37000E80001C0B901FC0120E06115710591F1BF
:10F380008EB38823E1F18530E1F18091E80083FDBF
:10F390003AC08091E80082FF06C08091E80082FFB9
:10F3A00024C080E008958091E80080FFE6CF80913E
:10F3B000F2009091F3006115710551F088309105CC
:10F3C00038F421912093F100615071090196F3CF37
:10F3D00021E0089709F020E08091E8008E77809383
:10F3E000E800CBCF2111CCCFD8CF8EB3882339F012
:10F3F000853039F08091E80083FFCFCF04C082E0F0
:10F40000089583E0089581E008958F708093E90066
:10F41000EBEEF0E0808181608083EDEEF0E0108221
:10F420006093EC0040838091EE00881F8827881F3E
:10F4300008950F931F93CF93DF93062FEC0110E0F5
:10F44000101771F19881992341F12C81E981FA819A
:10F450007B81892F8F70873010F080E022C02230AE
:10F4600010F056E001C052E028E030E040E02E17F6
:10F470003F0720F44F5F220F331FF9CF4295407FA3
:10F48000452B692F661F6627661F90E4799F9001C0
:10F490001124622BBADF882301F31F5F2596D0CF9A
:10F4A00081E0DF91CF911F910F91089580918302A8
:10F4B00087FD05C08091E80080FF0DC010C08091DD
:10F4C000E80082FD04C08EB38111F9CF08958091C8
:10F4D000E8008B7707C08EB38111ECCF089580913F
:10F4E000E8008E778093E80008958091E400909181
:10F4F000E50045E62091EC0020FF20C02091E800C7
:10F5000020FD20C02EB3222389F0253089F02091E0
:10F51000EB0025FD0FC02091E4003091E500281795
:10F52000390741F3415041F0C901E4CF82E0089529
:10F5300083E0089581E0089584E008952091E80033
:10F5400022FFE0CF80E008950F931F93CF93DF93C6
:10F5500049D050D0C8EDD0E088818F7788838881EA
:10F560008068888388818F7D8883E7EDF0E08081E3
:10F570008068808319BC1EBA1092810200EE10E0F0
:10F58000F80180818B7F808388818160888342E05D
:10F5900060E080E03ADFE1EEF0E080818E7F808302
:10F5A000E2EEF0E0808181608083808188608083EA
:10F5B000F80180818E7F8083888180618883DF91DC
:10F5C000CF911F910F910895E8EDF0E080818F7E3B
:10F5D0008083E7EDF0E080818160808381E080932B
:10F5E0008202B2CFE8EDF0E080818C7F80831092C0
:10F5F000E20008951092DA001092E10008951F923F
:10F600000F920FB60F9211240BB60F922F933F93C8
:10F610004F935F936F937F938F939F93AF93BF931A
:10F62000EF93FF938091DA0080FF1BC08091D80098
:10F6300080FF17C08091DA008E7F8093DA0080917E
:10F64000D90080FF0BC084E189BD86E189BD09B482
:10F6500000FEFDCF81E08EBB24D903C019BC1EBAC9
:10F6600021D98091E10080FF17C08091E20080FFE6
:10F6700013C08091E2008E7F8093E2008091E200CF
:10F6800080618093E2008091D80080628093D800EE
:10F6900019BC85E08EBBB2D18091E10084FF2EC001
:10F6A0008091E20084FF2AC084E189BD86E189BDA2
:10F6B00009B400FEFDCF8091D8008F7D8093D800E3
:10F6C0008091E1008F7E8093E1008091E2008F7E47
:10F6D0008093E2008091E20081608093E20080915B
:10F6E0008102882311F084E007C08091E30087FF46
:10F6F00002C083E001C081E08EBB80D18091E10037
:10F7000083FF26C08091E20083FF22C08091E10048
:10F71000877F8093E10082E08EBB1092810280910E
:10F72000E1008E7F8093E1008091E2008E7F8093E4
:10F73000E2008091E20080618093E20042E060E0BC
:10F7400080E063DE8091F00088608093F00056D105
:10F75000FF91EF91BF91AF919F918F917F916F91A9
:10F760005F914F913F912F910F900BBE0F900FBE65
:10F770000F901F9018951F920F920FB60F921124A1
:10F780000BB60F922F933F934F935F936F937F939B
:10F790008F939F93AF93BF93CF93EF93FF93C091BA
:10F7A000E900CF708091EC001092E9008091F000A8
:10F7B000877F8093F00078941DD01092E9008091AB
:10F7C000F00088608093F000C093E900FF91EF9112
:10F7D000CF91BF91AF919F918F917F916F915F91E9
:10F7E0004F913F912F910F900BBE0F900FBE0F9036
:10F7F0001F9018951F93CF93DF9300D0CDB7DEB73E
:10F80000E3E8F2E08091F100819382E0EB38F807C1
:10F81000C9F74DD88091E80083FFDCC09091830246
:10F8200080918402853009F465C030F4813059F14B
:10F8300068F0833041F1CEC0883009F49DC0893032
:10F8400009F4ACC0863009F0C5C075C0903881F0AD
:10F85000923809F0BFC0809187028F708093E900D1
:10F860009091EB0095FB992790F91092E90001C067
:10F8700090E08091E800877F8093E8009093F1000A
:10F880001092F10084C0292F2D7F09F0A3C092307F
:10F8900009F0A0C090918502911126C020918702A5
:10F8A0002F7009F497C02093E9009091EB0090FF2E
:10F8B0001BC0833021F48091EB00806213C08091E3
:10F8C000EB0080618093EB0081E090E0022E01C0AC
:10F8D000880F0A94EAF78093EA001092EA00809178
:10F8E000EB0088608093EB001092E9008091E800C3
:10F8F000877F50C091116EC0109185021F77809153
:10F90000E3008078812B8093E3008091E800877F7B
:10F910008093E800CBDD8091E80080FFFCCF8091F0
:10F92000E30080688093E300112311F083E001C0BD
:10F9300082E08EBB4FC09058923008F04BC0AE01B1
:10F940004F5F5F4F609187028091850290918602A0
:10F950000E945FF4009709F43DC02091E800277FE2
:10F960002093E800BC0189819A81F4DC8091E80051
:10F970008B778093E8002EC0903861F58091E80085
:10F98000877F8093E800809181028093F1008091CD
:10F99000E8008E778093E80089DD1CC091111AC0C1
:10F9A000909185029230B0F48091E800877F809337
:10F9B000E800909381027ADD80918102811104C078
:10F9C0008091E30087FF02C084E001C081E08EBB2C
:10F9D0000E9453F48091E80083FF0AC08091E80000
:10F9E000877F8093E8008091EB0080628093EB003A
:10F9F0000F900F90DF91CF911F9108950895CF93AD
:10FA00008EB38823A9F08091E9008F709091EC006B
:10FA100090FF02C090E801C090E0C92FC82B10925F
:10FA2000E9008091E80083FDE5DECF70C093E90036
:10FA3000CF910895CF93DF93EC018091E80083FF8D
:10FA400035C0888190E02091870230918802281784
:10FA5000390761F5809184028E3F79F08F3F31F54F
:10FA600080918302813211F58091E800877F809335
:10FA7000E8001CDD81E088AF19C080918302813AE3
:10FA8000A9F48091E800877F8093E8008091E800E6
:10FA900080FFFCCF8B8581508093F1008091E8003E
:10FAA0008E778093E800DF91CF9100CDDF91CF91E9
:10FAB0000895CF93DF93EC01FC013C968DE2DF01CA
:10FAC0001D928A95E9F782E08C83898761E0CE01F7
:10FAD0000196AFDC882331F061E0CE010696DF911C
:10FAE000CF91A7CC80E0DF91CF910895EF92FF9264
:10FAF0000F931F93CF93DF9300D0CDB7DEB78C0168
:10FB00008EB3843009F000C1F80186818F70809334
:10FB1000E9008091E80082FFBDC086818F708093EC
:10FB2000E9001A8219827801FCE0EF0EF11CAE01A7
:10FB30004F5F5F4F6FE070E0C701C5DBF8018530B4
:10FB400021F480AD882399F3A5C084859585A68589
:10FB5000B78585359345A244B34461F4F801918D8E
:10FB60008385981738F4808D8F7121F4828D8150B0
:10FB7000803180F08091EB0080628093EB00F8018F
:10FB800081818F708093E9008091EB008062809387
:10FB9000EB0080C01A8219827801FBE1EF0EF11CA4
:10FBA000F801628D70E0AE014F5F5F4FC7018BDBE4
:10FBB000853029F4F80180AD882391F36BC08091E2
:10FBC000E8008B778093E800F801808D87FF04C000
:10FBD00081818F708093E900C8010E945BF491E0FD
:10FBE0009827F80197AB45E553E562E473E543A731
:10FBF00054A765A776A7408951896289738947A769
:10FC000050AB61AB72AB448955896689778943AB48
:10FC100054AB65AB76AB811109C0452B462B472B06
:10FC200029F08091EB0080628093EB00F8018681DF
:10FC30008F708093E9008091EB00F80185FF04C08C
:10FC400080AD8823C1F326C081818F708093E90045
:10FC50008091EB0085FF05C0F80180AD8823C1F3DA
:10FC600019C01A8219827801FBE2EF0EF11CAE0175
:10FC70004F5F5F4F6DE070E0C701DEDA853029F439
:10FC8000F80180AD882399F305C08091E8008E7754
:10FC90008093E800F80180AD8823B1F126812F70B0
:10FCA00081E090E0AC0102C0440F551F2A95E2F7B5
:10FCB0004093EA001092EA0021812F70022E01C0C9
:10FCC000880F0A94EAF78093EA001092EA0086818E
:10FCD0008F708093E9008091EB0080618093EB004E
:10FCE0008091EB0088608093EB0081818F7080931E
:10FCF000E9008091EB0080618093EB008091EB0044
:10FD000088608093EB0010AE0F900F90DF91CF9141
:10FD10001F910F91FF90EF900895F999FECF92BD3A
:10FD200081BDF89A992780B50895262FF999FECFBD
:10FD300092BD81BDF89A019700B4021639F01FBA3E
:10FD400020BD0FB6F894FA9AF99A0FBE0895F89468
:02FD5000FFCFE3
:10FD52000100834000000104400000010100000096
:10FD62000000000000000000000000000000000091
:10FD72000000000000000000000000000000000081
:10FD82000000000000000000000070000000000001
:10FD9200000A000000000000000000004C5546412F
:10FDA20020424F4F542020080000000000000000B5
:10FDB2000000000000000000000000004146004C6E
:10FDC200004100530048000F00262E004200490067
:10FDD2004E0000000000000000000000464C4153AD
:10FDE2004820202042494E00000000000000000090
:10FDF200000020084E12020000E8010041450045C3
:10FE020000500052004F000F00144D002E0042001F
:10FE120049004E000000000000000000454550521D
:10FE22004F4D202042494E0000000000000000001B
:10FE3200000020084E123F00FF0F000009022000C0
:10FE42000101008032090400000208065000070583
:10FE5200830240000507050402400005120110015B
:10FE620000000008EB0345200100000000010080B3
:10FE720000021F0000004C55464100000000426F86
:10FE82006F746C6F61646572000000000000302EB8
:10FE92003030EB3C906D6B646F736673000002044C
:10FEA20001000210001C01F801001C000400000007
:10FEB200000000000000000029785634124C55461C
:10FEC2004120424F4F5420204641543132202020BD
:10FFA000B4C8C7C8DAC8E8C8EDC8F2C8F8C8089528
:08FFB0000895089508950895D5
:10FFE000DFCFDFCFDFCFDFCFDFCFDFCFDFCFDFCFA1
:08FFF000DFCFDFCFDFCFDFCF51
:08FFF80000F0010030DFFBDC2A
:040000031000F000F9
:00000001FF
